S02B0000433A2F576F726B2F736F6674776172652F4F70656E424C542F5461726765742F44656D6F2F41524DEF
S11300006C0D0020F1000000E5120000E512000074
S1130010E5120000E5120000E5120000E512000000
S1130020E5120000E5120000E5120000E5120000F0
S1130030E5120000E5120000E5120000E5120000E0
S1130040E5120000E5120000E5120000E5120000D0
S1130050E5120000E5120000E5120000E5120000C0
S1130060E5120000E5120000E5120000E5120000B0
S1130070E5120000E5120000E5120000E5120000A0
S1130080E5120000E5120000E5120000E512000090
S1130090E5120000E5120000E5120000E512000080
S11300A0E5120000E5120000E5120000E512000070
S11300B0E5120000E5120000E5120000E512000060
S11300C0E5120000E5120000E5120000E512000050
S11300D0E5120000E5120000E5120000E512000040
S11300E0E5120000E5120000E5120000E512000030
S11300F02949072291438D4628482949294A00F075
S113010039F8294829492A4A00F034F829482A4963
S11301102A4A00F02FF82A482A492B4A00F02AF8E4
S11301202A482B492B4A00F025F82B482B492C4A06
S113013000F020F82B482C49002200F026F82B4828
S11301402B49091A082903DB0022026004300160EC
S11301501C481D49884205D00268043003B4904706
S113016003BCF7E700208646EC4600200021214A24
S11301709047FEE7884207D0521A05D00378013031
S11301800B700131013AF9D17047884202D00270F4
S11301900130FAE7704700006C0D0020482200008F
S11301A00000002001000020F8010000F801000018
S11301B01C1D000048220000000000200000002058
S11301C01C1D00001C1D00001C1D00001C1D000047
S11301D01C1D00001C1D00001C1D00001C1D000037
S11301E04822000004000020EC040020EC0400205D
S10B01F06C050020A5120000BB
S11301F820F08053A3F58012013A012A10B559D989
S11302082D4A934256D002F58072934252D002F599
S1130218007293424ED002F1005202F59842904285
S113022848D000F16042013A1F2A04D8234921FA30
S113023802F2D2073ED4224A93423BD020F48011E2
S11302488032914236D020F00052402A32D0B0F1A8
S1130258102F2FD01B4CA1422CD0B0F1101F29D045
S1130268A4F57C54A04225D004F58074A04221D082
S1130278A4F5F874A2421DD01034A2421AD004F591
S11302887F2404F6E874A04214D000F17044013CC1
S1130298012C0FD90C4CA1420CD0B0F1202F09D05D
S11302A80A49884206D0082A04D009481B1A584229
S11302B8584110BD012010BD000110000B800080C2
S11302C880000020004000100400001001001020ED
S11302D80010100010B50446FFF78AFF20B94FF448
S11302E8FC71084801F03EFB074B220F53F822101B
S11302F8A2B20B68C4F3044402FA04F41C430C606D
S113030810BD00BF781D0000E41D000001387FF413
S1130318FDAF7047F8B5424B0246196811F0E04F3B
S113032805D019683F4B0B40B3F1805F01D1002A17
S113033874DB3D493D4C0D68266825F4800343F47D
S1130348006346F40060AF070B60206001D597078F
S113035803D5ED0714D5D70712D462F00305002896
S113036803EA0503B4BF06F0300003F03000302878
S11303780B600CBF4FF480504FF40020FFF7C6FF0A
S113038843F2F07023F45F53104023F0300340EA43
S11303980305274B27483340104043F400630343C5
S11303A8D00000F04000244E03434FF0400737606C
S11303B84FF010004BBF23600D600D602360FFF702
S11303C8A5FF25F0F8601D4D20F0030015402843D3
S11303D823F0FC5302F0FC552B43550041BF184D44
S11303E823F48003154040F480004CBF2B4323F0D2
S11303F8804317050BD4134D4FF400422E6876063C
S113040801D4013AFAD120F4006023F400630860AF
S113041823601020BDE8F840FFF778BFF8BD00BF9F
S113042800E00F400000FF7060E00F4070E00F40F4
S11304388FDFFF7F3020008058E00F400300C007A3
S11304480000404050E00F40664BF0B51968103387
S11304581B68002B13DA03F07002202A45D003D856
S1130468E2B1102A20D0B6E0602A00F0B680702AE3
S11304786DD0302A40F0AF8047F2305069E001F087
S11304883002102A10D001D842B1A4E0202A2CD07E
S1130498302A40F0A08047F230505DE0524AC1F360
S11304A8841052F820004FE0504A106810F0E04FD2
S11304B83FD014684E482040B0F1805F39D01468AA
S11304C84B4820404B4CA04203D1126892B2022AF6
S11304D831D04648464A04682240474CA2422CD1AF
S11304E80068464C82B246481FE0404A106810F043
S11304F8E04F24D014683E482040B0F1805F1ED0FD
S113050814683B4820403B4CA04203D1126892B285
S1130518022A16D03548364A04682240364CA2428C
S113052811D10068374C82B23748002A18BF2046D8
S11305380AE0364808E0324806E0304804E0344827
S113054802E0314800E02F48002B05DA01E04FF4BF
S1130558004013F4006F01E011F4006F23D12D4A19
S1130568224E1568326805F01F0412F0E04F4FEA76
S11305785512C2F3080205D037681D4E3E40B6F145
S1130588805F03D102325043023402E05043013405
S11305986400B0FBF4F06E0448BF40082D0448BF63
S11305A8800841F480014C021AD5002B0DDA590059
S11305B805D51A0503D44000C3F3865301E0C3F3F9
S11305C8C5530133B0FBF3F0F0BDC1F3C35101319E
S11305D8B0FBF1F0F0BD0020F0BD4FF48000B8E7A7
S11305E8F0BD00BF60E00F401C1D000000E00F409C
S11305F80000FF7000000110000003100024F40044
S1130608001BB70000093D00C0C62D00C0E1E4008E
S11306187038390064E00F40462810B5044605D9FF
S11306284FF4D571184801F09DF90EE0042804D15F
S1130638164A136843F4803305E0052805D1134AA4
S1130648136843F40033136010BD062C04D10F4A19
S1130658136843F48023F6E70F2C04D10C4A13687B
S113066843F00203EFE7A4F110021F2A03D8012381
S11306789340084AE7E72F2C05D90123303C03FAB5
S113068804F4054B1C6010BDF01D000024ED00E0CF
S113069810E000E000E100E004E100E0462810B5C5
S11306A8044605D94FF4F771184801F05BF90EE0D8
S11306B8042804D1164A136823F4803305E0052876
S11306C805D1134A136823F40033136010BD062CB4
S11306D804D10F4A136823F48023F6E70F2C04D1BE
S11306E80C4A136823F00203EFE7A4F110021F2A4F
S11306F803D801239340084AE7E72F2C05D901239F
S1130708303C03FA04F4054B1C6010BDF01D0000D6
S113071824ED00E010E000E080E100E084E100E086
S113072820F44053B3F1402F13D00B4A934210D016
S1130738A2F5503293420CD002F56032934208D0AD
S1130748064B984205D003F50C33C31A5842584156
S113075870470120704700BF0080054000D0034067
S113076870B505460C461646FFF7DAFF18B9E421BA
S11307780E4801F0F7F8022E03D9E6210B4801F0E0
S1130788F1F8D5F80034F0074CBF2343A34305F52B
S113079880621360D5F82024B10705F584634CBF43
S11307A8144322EA04041C6070BD00BF5E1E0000EE
S11307B82DE9F04104460D4617461E46FFF7B0FFE3
S11307C820B94FF4DD713B4801F0CCF87B1E012BB6
S11307D804F5A06808D927F00803042B16D04FF4B1
S11307E8DF71344801F0BEF8082E09D0A6F10903D8
S11307F8042B05D926B140F2C5112E4801F0B2F8F0
S1130808FB0705D5D4F800352B4305E0082EEDD1B8
S1130818D8F8003023EA0503C8F80030D4F80435C2
S1130828B80704F204524CBF2B43AB431360D4F80B
S11308380835790704F5A1624CBF2B43AB43136019
S1130848D4F81835380704F5A3624CBF2B43AB43DF
S11308581360D4F80C35F10704F20C524CBF2B4347
S1130868AB431360D4F81035B70704F5A2624CBF44
S11308782B43AB431360D4F81435700704F21452B5
S11308884CBF2B43AB431360D4F81C35310704F237
S11308981C524CBF2B43AB431360D4F8283504F5E2
S11308A8A5620EB91D4301E023EA05051560BDE8FC
S11308B8F08100BF5E1E000070B504460D46FFF7C8
S11308C82FFF20B94FF46471074801F04BF829460B
S11308D820460222FFF744FF29462046BDE870401F
S11308E808230422FFF764BF5E1E000070B50446A7
S11308F80D46FFF715FF20B940F21F51074801F0D4
S113090831F8294620460222FFF72AFF29462046C5
S1130918BDE8704008230122FFF74ABF5E1E0000AD
S1130928C0F3090310B504461BB18421094801F03A
S113093819F8094B01221A60084A43F8144C0C3B75
S11309481A601A689207FCD4054B186840F3000033
S113095810BD00BFC71E000014D00F40020042A4FF
S11309680CD00F402DE9F041044688070D46164681
S113097803D0C821294800F0F5FFB10703D0C921E5
S1130988264800F0EFFF264B01221A6003F58C532A
S11309980C331B68DA0709D4224A23462D1B224F3D
S11309A8DFF89CE0DFF88CC0904623E01F4A1E491C
S11309B896461F481F4F56B325F07F030B60C4EBC0
S11309C8050804EB080515F07C0C01D103683BB954
S11309D836B1194B54F8045B043E43F80C50F0E765
S11309E81760DEF80030DB07FBD4E4E7D8F8001022
S11309F8C907FBD4F11ACC4205EB030007D03860D1
S1130A0853F8041BCEF80010C2F800C0EEE70B4BF5
S1130A18186840F30000BDE8F08100BFC71E00005D
S1130A2814D00F4008D00F4000D00F4020D00F4002
S1130A3830D00F40010042A400D10F400CD00F4029
S1130A4804D00F40064B20F480529A4205D003F597
S1130A580053C31A5842584170470120704700BFD9
S1130A6800C0004010B50446FFF7ECFF20B94FF46E
S1130A78CF71074800F076FFE36A43F01003E3629E
S1130A88236B43F4407343F00103236310BD00BF99
S1130A98341F000010B50446FFF7D4FF20B94FF403
S1130AA8DF71084800F05EFFA3691B07FCD4E36A02
S1130AB823F01003E362236B23F4407323F0010350
S1130AC8236310BD341F0000F8B505460C461746CD
S1130AD81E46FFF7B7FF20B940F20D112C4800F06D
S1130AE841FF27B94FF48771294800F03BFF294B90
S1130AF81A6812F0E04F1DD01968274A0A40B2F16B
S1130B08805F17D01968244A0A4024498A4203D1CD
S1130B181B689BB2022B0DD01E4A1F4B11680B4059
S1130B281F498B4208D113689BB2002B14BF0823BA
S1130B38102302E0102300E008237B43A34204D9D6
S1130B4840F20F11124800F00DFF2846FFF7A2FFEC
S1130B58B4EB071F38BF7F084FEAC404B4FBF7F4AB
S1130B682B6B04F1010435BF43F0200323F0200369
S1130B782B632B63E3096B62C4F345040023AC6263
S1130B882846EE62AB61BDE8F840FFF76BBF00BFD3
S1130B98341F000000E00F400000FF700000011047
S1130BA80000031010B50446FFF74CFF20B940F2CB
S1130BB8E931044800F0D6FEA06980F02000C0F3B3
S1130BC8401010BD341F000010B50446FFF73AFF6B
S1130BD820B940F20941054800F0C4FEA369DB06C8
S1130BE854BF20684FF0FF3010BD00BF341F000011
S1130BF838B504460D46FFF725FF20B940F25B419E
S1130C08044800F0AFFEA3699B065ABF0120256083
S1130C18002038BD341F0000064B20F480529A424D
S1130C2805D003F50053C31A5842584170470120B0
S1130C38704700BF00000440094B98420BD003F5ED
S1130C488053984209D0A3F5005398420CBF37202B
S1130C584FF0FF307047382070473920704700BF85
S1130C680010044082B0016000230193019B042B0F
S1130C7802DC019B0133F8E702B0704773B50646FE
S1130C8820F47F6020F00F00FFF7D6FF431C0546D1
S1130C9803D1F9210F4800F065FE0F4B01221C68AF
S1130CA8A5F1300302FA03F31C4002D02846FFF7EB
S1130CB8F5FC336800230193019B042B02DC019BA0
S1130CC80133F8E7366814B12846FFF7A5FC304627
S1130CD802B070BDA01F000004E100E0F8B50446AE
S1130CE8FFF79AFF20B940F2D911214800F03AFEE3
S1130CF801212046FFF7B6FF04F120052846FFF737
S1130D08BDFF10F40042F9D104F12407B02138469C
S1130D18FFF7A8FF04F134001146FFF7A3FF04F11D
S1130D2838001146FFF79EFF01262846FFF7A6FF65
S1130D380204FAD4314628460136FFF793FF212EE0
S1130D48F3D10C213846FFF78DFF01262846FFF71B
S1130D5895FF0304FAD4314628460136FFF782FF8B
S1130D68212EF3D1201DBDE8F840FFF787BF00BF4F
S1130D78A01F000010B50446FFF74EFF20B940F24B
S1130D883A21064800F0EEFD2046FFF777FF20F0F1
S1130D9801012046BDE81040FFF764BFA01F000012
S1130DA870B506460C46FFF737FF20B94FF4597162
S1130DB8314800F0D7FD24B940F265312E4800F0DF
S1130DC8D1FD2368023B0E2B04D940F26B312A482B
S1130DD800F0C8FD6368013B072B04D94FF45C712C
S1130DE8254800F0BFFDA368013B032B04D940F25A
S1130DF87531214800F0B6FDE368013BB3F5806F17
S1130E0804D340F27B311C4800F0ACFD3046FFF7B8
S1130E1835FF054640F041013046FFF723FF63687C
S1130E28E168013B1B0303F4E04223680139013BF9
S1130E381B0203F47063134301F03F010B43A168E1
S1130E4806F10C0001398901C9B21943FFF70AFFF9
S1130E58E16806F118000139C1F38311FFF702FFB5
S1130E68EB0754BF25F0400125F041013046BDE8A9
S1130E787040FFF7F7BE00BFA01F000038B5054655
S1130E880C46FFF7C9FE20B940F29251194800F008
S1130E9869FD032C2AD8DFE804F0020D151D04357A
S1130EA82846FFF7EBFE6FF01F0102462846FFF7BE
S1130EB8D9FE1CE005F58070FFF7E0FE044605F551
S1130EC882700EE005F59070FFF7D8FE044605F52C
S1130ED8927006E005F5B070FFF7D0FE044605F5FC
S1130EE8B270FFF7CBFE44EA004200E0002210464D
S1130EF838BD00BFA01F00002DE9F04F85B006469D
S1130F08894690461C46FFF787FE20B940F25F6188
S1130F18734800F027FD09F1FF331F2B04D94FF460
S1130F28CC616F4800F01EFD042C04D940F26661C0
S1130F386B4800F017FD06F1200A5046FFF79EFEA5
S1130F480304FAD4D8F80010B1F5006F36BFD8F806
S1130F5808304FF0010CC3F3800C042C00F2BD8060
S1130F68DFE804F01C03070D180000234FF4807514
S1130F7801E000231D469E461A461F4615E000233D
S1130F884FF480554FF4005E41F6FF724FF6FF7739
S1130F98D3240BE001234FF4905502E001234FF4CE
S1130FA88075002217464FF4005E9324D8F8080091
S1130FB810F0080F0DD0D8F80420BCF1000F03D0AE
S1130FC897B2C2F30C4204E067469200C2F30C02E3
S1130FD892B200F0280BBBF1280F00F0180B08BFE1
S1130FE842F40042BBF1180F08BF42F4804210F0EB
S1130FF8380F18BFD32444F0200418BF45F4805593
S11310080294BCF1000F08D08CB20094C1F30C44D4
S113101844EA0E0444F4404408E08C00C4F30C048D
S113102844EA0E0444F40044CDF800C0D8F80CB0E7
S11310380BF00F010D4381055CBF45F08005ADB28F
S1131048C10748BF45F40065810748BF45F480657A
S11310582BBB029906F12400FFF704FE394606F17A
S11310682800FFF7FFFD06F12C001146FFF7FAFDF3
S1131078009906F13000FFF7F5FD214606F134002A
S1131088FFF7F0FD294606F13800FFF7EBFD50465F
S113109809F03F0105B0BDE8F04FFFF7E3BDD8F80C
S11310A810300020019306F13C038345D1DD00F1A3
S11310B801080199C34511F800C0C2BF11F808E03E
S11310C800F102084CEA0E2C184661460393FFF718
S11310D8C9FD039B40460433E7E705B0BDE8F08F3C
S11310E8A01F00002DE9F74F05460F4614461E467B
S11310F8FFF792FD20B940F2C171664800F032FC56
S11311087B1E1F2B04D940F2C271624800F02AFCEE
S1131118002E05F184090CBF73217B21484605F193
S1131128800807F03F07FFF79DFD39464046FFF763
S113113899FD4046FFF7A2FD0204FAD405F18800A0
S1131148FFF79CFD824605F18C00FFF797FD834667
S113115805F19000FFF792FD019005F19400FFF767
S11311688DFD064605F19800FFF788FD82B212F45A
S1131178807FB1B203D18B0403D4002302E08B0433
S1131188FBD4402311F48041A3600DD04FEA064EEE
S1131198414EBDF804300EEA060633432360A368C3
S11311A843F00403A36002E0C6F38A0626605304EE
S11311B842BFA36843F48073A360D60427D5A36809
S11311C859B135494FEA0B4631401FFA8AFA41EAC8
S11311D80A0161606FF0604604E040F2FF76CBF3E9
S11311E88A016160B14201D1590602D443F008036F
S11311F8A3601BF4004F1EBFA36843F02803A36039
S11312081BF4804F1EBFA36843F01803A3601605A0
S113121842BFA36843F00103A360510542BFA3681A
S113122843F00203A36002042ED5A66800F00F0A57
S113123816F04006C4F80CA008D048460421FFF76D
S113124811FD39464046FFF70DFD13E0D4F810B000
S11312589C35B245F1DD2846FFF710FD731C9A450D
S11312680BF80600C2BF000A0BF80300B31C0435D0
S11312781E46EEE74046FFF701FD0304FAD4A368CF
S113128843F08003A36001E00023E36003B0BDE8FA
S1131298F08F00BFA01F00000000FF1F08B50B4817
S11312A8FFF738F80A48FFF715F803214FF04020F4
S11312B8FFF71CFB0748FFF70DF803210648FFF763
S11312C8FBFA00F07FFB00F08CFBFCE78003C00115
S11312D80100002008000020007000403821014867
S11312E800F040BB0B20000072B6704762B670472E
S11312F8FFF7FABF10B500F0D0F9A0B100F0AAFBCF
S113130800F0E8F900F0CBF9074B20F0604020F03A
S11313187F00186000F0C3F94468FFF7E7FF23462D
S1131328BDE81040184710BD08ED00E0013A70B55B
S11313384D1E5618441AB54205D015F8013F635599
S113134800F0B5FBF7E770BDF8B505460A4E002472
S11313580C2700F0ACFB07FB04F39959A94206D803
S113136833445A680A44954201D2187AF8BD0134C4
S1131378102CEED1FF20F8BD902000002DE9F34198
S113138805460068FFF7E0FFFF2801D1002019E0B7
S11313980024261D2F68AB5904EB0708019300F0BD
S11313A886FB042241460DEB0200FFF7DBFA002816
S11313B8ECD1E259019B9A42E8D1B6F5007F344654
S11313C8E7D1012002B0BDE8F081000038B5114B27
S11313D8044698420D4606D0B1F5004F05D0FFF7F4
S11313E8CDFF18B911E00C4C00E01C46C5F3080306
S11313F85BB923689D420AD020464FF4007240F836
S1131408045B2946FFF792FF01E0002038BD20461F
S113141838BD00BF04000020080200202DE9F8436D
S11314289846036821F4FF76013304460D461746AF
S113143826F0010606D140F8046B4FF400723146D9
S1131448FFF774FF23689E4208D020463146FFF711
S1131458BDFF044610B90020BDE8F883B9462368E7
S113146806F50076ED1A2544043500F020FB231D0B
S1131478EB1AB3F5007F07D320463146FFF7A6FFE2
S113148804460028E7D0051D19F8013B05F8013B7F
S1131498C9EB0803DF42E8D10120BDE8F883000066
S11314A8034A4FF0FF331360024A1360704700BFCA
S11314B80802002004000020FFF7F2BF70B50446BC
S11314C80D461646FFF740FFFF2815D0681E204436
S11314D8FFF73AFFFF280FD024F4FF7323F001032A
S11314E8B3F5004F32462B462146BDE870400CBF89
S11314F802480348FFF792BF002070BD0400002093
S1131508080200202DE9F8430C460646FFF71CFFA5
S11315180546601E3044FFF717FF8542074602D987
S11315280020BDE8F8832B1FDBB2FA2BF8D8132868
S1131538F6D8244E00244FF00C0900F0B8FA09FB41
S113154804631A7ADFF87C80AA4201D11E6804E099
S11315580134102CF1D14FF0FF3600240C2500F093
S1131568A6FA05FB04831A7ABA4201D11C6804E07E
S11315780134102CF3D14FF0FF3400254FF00C093F
S113158800F095FA09FB05831A7ABA4201D15B681F
S113159803E00135102DF3D10023A41B2344C3F326
S11315A88F240025ABB29C4209D900F080FA06EBDF
S11315B88520FFF7B5F901350028F3D0B0E70120FD
S11315C8BDE8F883902000000F4B07B51A68013274
S11315D816D09A68596848F2F0001144DA68114440
S11315E81A6911445A6911449A691144DA698B18C1
S11315F85B4202AA42F8043D0421FFF75FFF00E0C2
S1131608012003B05DF804FB040000204FF40043FC
S11316181A6848F204031B68134448F20802126863
S1131628134448F20C021268134448F21002116879
S113163848F2140212680B441A4448F218031B684F
S1131648134448F2F0021268D3420CBF0120002070
S1131658704700000A4808B50368013305D10948F2
S11316680368013306D1012008BDFFF787FE00286F
S1131678F5D108BDFFF782FE003018BF012008BD70
S113168804000020080200204FF400407047FFF7D0
S113169813BFFFF713BFFFF735BFFFF7B7BFFFF758
S11316A8F3BF08B5FFF790FF18B1BDE80840FFF78E
S11316B8D1BF08BD4CF24F31044B00221A60596067
S11316C805219A601960024B1A60704710E000E027
S11316D80C040020014B00221A60704710E000E05F
S11316E8044B1B68DB0341BF034A136801331360CF
S11316F8704700BF10E000E00C04002008B5FFF7B5
S1131708EFFF014B186808BD0C04002010B507480A
S1131718FEF7E0FDFEF798FEBDE8104001466023A1
S11317284FF461420248FFF7CFB900BF010000102F
S113173800C00040402970B506460C4603D95B2119
S1131748174800F00FF921461648FFF751FA30B14F
S11317581448FFF727FA30B900F0A9F9F8E75F2130
S11317680F4800F0FFF83546A4B2AB1B9BB2A34266
S11317780FD200F09CF915F8011B0A48FFF738FA54
S113178840B10848FFF70EFA0028EED100F08FF9AF
S1131798F7E770BD6821024800F0E4F8E5E700BF08
S11317A85021000000C00040F8B51F4D07462C78B2
S11317B8A4B91E48FFF708FA421C01D1002430E0FE
S11317C81B4BC0B218700028F8D0FFF797FF194BCD
S11317D81860194B1C7001232B7022E0164C134817
S11317E82678FFF7F1F9431C06F1010610D01049D9
S11317F82378885501330A78DBB29A422370DDD105
S113180801313846FFF792FD00232B70012408E0CC
S1131818FFF774FF074B1B6864339842CED9002442
S11318282C702046F8BD00BF5204002000C00040C0
S1131838100400205404002051040020F0B5264868
S113184887B0FEF747FD2548FFF748FA04230393BA
S1131858102340F2A4641E460193002508225F1C4D
S1131868E2B1B818B4FBF0F14139C9B20A2913D866
S1131878B6FBF0F1414310290ED1029205B1019350
S11318881023B3FBF0F0032A049001A9134898BF6E
S11318980392FFF785FA0BE0013AE1E7013BA4F173
S11318A864044FF00105D9D18B210D4800F05AF892
S11318B80A48FFF75FFA40F26763019340F2FF7347
S11318C8029308230393049301AA022301210348E2
S11318D8FFF712FB07B0F0BD000110000000044040
S11318E8C721000030B5044687B00D4610480121D1
S11318F8FFF7C4FA820703D5AE210E4800F032F888
S113190840F2E17301AA01930221002308480393DA
S113191804950594FFF7F0FA01210548FFF7AEFA9C
S1131928044600F0C4F8A307F6D407B030BD00BFDE
S113193800000440C721000010B5022186B0044607
S11319480748FFF79BFA10F0010007D00123044869
S113195801AA19460594FFF7C5FB012006B010BD7E
S11319680000044008B500F0A2F8FCE710B500F048
S11319789BF8012811D0094C2378012B0DD1FFF7CE
S1131988BDFE074B1B6803F5FA73984205D3002381
S11319982370BDE81040FFF7ADBC10BD580400200B
S11319A85C04002008B5054B01221A70FFF7A6FE57
S11319B8034B1860BDE80840FFF7D8BF580400205F
S11319C85C04002008B5FFF793FC00F06FF8FFF7FC
S11319D871FEFFF75CFE00F00FF8BDE80840FFF762
S11319E8E1BF08B500F063F8FFF77AFE00F014F8D9
S11319F8BDE80840FFF7BABF10B5064C00F062F81E
S1131A08FFF71CFF01232370FFF780FE00232370D8
S1131A1810BD00BF0000002008B50C48FFF78CFF7C
S1131A28012804D10A4B1870084800F069F80748DF
S1131A38FFF7BAFE012807D1054B00221A700348A4
S1131A48BDE8084000F05CB808BD00BF6004002091
S1131A5800000020704700000A4B70B51A7806464B
S1131A68012A0D461C4602D1C9B2FFF73BFF237871
S1131A781BB9E9B23046FFF75DFEBDE8704000F0DF
S1131A8837B800BF00000020044B1B78013BDBB2D1
S1131A98022B9ABF024AD05C402070470000002005
S1131AA83D220000FFF7F0BF00F01AB870477047F6
S1131AB8034BFE22DA7002221871A3F844207047FF
S1131AC8A0040020054B00221A709A6483F843206E
S1131AD8A3F844209A705A70704700BFA0040020ED
S1131AE8024B1878003018BF01207047A00400206A
S1131AF8024B002283F84320704700BFA004002053
S1131B08F8B503780546FF2B804C19D1002201252E
S1131B18E37010232371627062712570FFF7C2FFAE
S1131B28A071FFF7B1FFE071FFF7AEFF0823000AC9
S1131B3820726572A572A4F84430FFF7A8FDCEE0C0
S1131B482678012E40F0E080F32B53D01ED8CF2BFB
S1131B5800F0B98005D8C92B7FD0CC2B00F0BA800F
S1131B68BAE0D12B00F0A980C0F08980D22B40F0D4
S1131B78B3800025FF23E37025716571FFF792FF99
S1131B88E571A07125726572072393E0FA2B46D09C
S1131B980AD8F52B11D019D3F62B40F09D80FF23DA
S1131BA8E3704368A36492E0FD2B47D0FE2B50D02A
S1131BB8FC2B40F0918000208FE0FFF773FF6A78D8
S1131BC8904201DC222088E0A16C07E0FFF76AFF5D
S1131BD86B789842F6DD6968A1646A78201DFFF77E
S1131BE8A5FBFF23E3706B78A26C1344A3646B78A2
S1131BF801335FE0FF23E370A26C416800231144C2
S1131C088A4204D012F8010B0344DBB2F8E7C4F8A3
S1131C1807300123237100236371A3710CE0FF23B0
S1131C28E3703B4B0722A364002323716371A37100
S1131C38E27123726372A37208233BE0FF23627884
S1131C48E37000232371A371E37123726271062385
S1131C5830E000232370637037E0A76CFFF722FF9E
S1131C686A1C411E3846FFF714FD98B3FF23E3703E
S1131C78FFF718FFA36C01381844A06427E0FFF7A6
S1131C8811FF6B78013898429CDDFF23E370A4F8B8
S1131C984460697819B9FFF704FD00BB1AE0AA1C6F
S1131CA8A06C1A4EFFF7F5FCA0B16B78B26C134424
S1131CB8B36414E0A4F8443011E04168A06CFFF761
S1131CC8EAFC10B906E0FFF715FBFF23E370A4F85C
S1131CD8446004E0312000E02020FFF7E9FE94F896
S1131CE84330012B02D11020FFF7E2FEB4F944106F
S1131CF80648002908DD012380F8433089B20330FF
S1131D08BDE8F840FFF7A8BEF8BD00BFA004002056
S1071D184022000061
S1131D1C40420F0000201C0080841E00008025001F
S1131D2C999E36000040380000093D0000803E00BA
S1131D3C00004B00404B4C0000204E00808D5B009B
S1131D4C00C05D000080700000127A0000007D006D
S1131D5C80969800001BB7000080BB00C0E8CE0042
S1131D6C647ADA000024F4000000FA00433A2F5796
S1131D7C6F726B2F736F6674776172652F4F70651A
S1131D8C6E424C542F5461726765742F44656D6FA9
S1131D9C2F41524D434D335F4C4D33535F454B5F95
S1131DAC4C4D3353383936325F43726F7373776FDC
S1131DBC726B732F426F6F742F6964652F2E2E2FE5
S1131DCC6C69622F6472697665726C69622F7379BF
S1131DDC7363746C2E63000000E10F4004E10F4048
S1131DEC08E10F40433A2F576F726B2F736F667471
S1131DFC776172652F4F70656E424C542F5461722B
S1131E0C6765742F44656D6F2F41524D434D335F9D
S1131E1C4C4D33535F454B5F4C4D3353383936324D
S1131E2C5F43726F7373776F726B732F426F6F7440
S1131E3C2F6964652F2E2E2F6C69622F647269765C
S1131E4C65726C69622F696E746572727570742E2A
S1131E5C6300433A2F576F726B2F736F66747761FD
S1131E6C72652F4F70656E424C542F5461726765C6
S1131E7C742F44656D6F2F41524D434D335F4C4D60
S1131E8C33535F454B5F4C4D3353383936325F43D4
S1131E9C726F7373776F726B732F426F6F742F69DA
S1131EAC64652F2E2E2F6C69622F647269766572AD
S1131EBC6C69622F6770696F2E6300433A2F576FFA
S1131ECC726B2F736F6674776172652F4F70656ECA
S1131EDC424C542F5461726765742F44656D6F2F97
S1131EEC41524D434D335F4C4D33535F454B5F4C27
S1131EFC4D3353383936325F43726F7373776F7265
S1131F0C6B732F426F6F742F6964652F2E2E2F6C99
S1131F1C69622F6472697665726C69622F666C6192
S1131F2C73686C69622E6300433A2F576F726B2F80
S1131F3C736F6674776172652F4F70656E424C5483
S1131F4C2F5461726765742F44656D6F2F41524D28
S1131F5C434D335F4C4D33535F454B5F4C4D3353C3
S1131F6C383936325F43726F7373776F726B732FBA
S1131F7C426F6F742F6964652F2E2E2F6C69622F3C
S1131F8C6472697665726C69622F756172746C69BE
S1131F9C622E6300433A2F576F726B2F736F667404
S1131FAC776172652F4F70656E424C542F54617279
S1131FBC6765742F44656D6F2F41524D434D335FEC
S1131FCC4C4D33535F454B5F4C4D3353383936329C
S1131FDC5F43726F7373776F726B732F426F6F748F
S1131FEC2F6964652F2E2E2F6C69622F64726976AB
S1131FFC65726C69622F63616E6C69622E63004357
S113200C3A2F576F726B2F736F6674776172652FEB
S113201C4F70656E424C542F5461726765742F4433
S113202C656D6F2F41524D434D335F4C4D33535FB0
S113203C454B5F4C4D3353383936325F43726F73B3
S113204C73776F726B732F426F6F742F6964652F84
S113205C2E2E2F2E2E2F2E2E2F2E2E2F536F75729B
S113206C63652F41524D434D335F4C4D33532F43D6
S113207C726F7373776F726B732F766563746F7291
S113208C732E630000800000002000000400000098
S113209C00A00000002000000500000000C00000AB
S11320AC002000000600000000E0000000200000FA
S11320BC07000000000001000020000008000000E0
S11320CC0020010000200000090000000040010075
S11320DC002000000A000000006001000020000045
S11320EC0B00000000800100002000000C00000028
S11320FC00A00100002000000D00000000C0010041
S113210C002000000E00000000E001000020000090
S113211C0F0000000000020000800000100000000E
S113212C0080020000800000110000000000030089
S113213C00800000120000000080030000800000FA
S113214C13000000433A2F576F726B2F736F667432
S113215C776172652F4F70656E424C542F546172C7
S113216C6765742F44656D6F2F41524D434D335F3A
S113217C4C4D33535F454B5F4C4D335338393632EA
S113218C5F43726F7373776F726B732F426F6F74DD
S113219C2F6964652F2E2E2F2E2E2F2E2E2F2E2EA2
S11321AC2F536F757263652F41524D434D335F4C02
S11321BC4D33532F756172742E6300433A2F576F4E
S11321CC726B2F736F6674776172652F4F70656EC7
S11321DC424C542F5461726765742F44656D6F2F94
S11321EC41524D434D335F4C4D33535F454B5F4C24
S11321FC4D3353383936325F43726F7373776F7262
S113220C6B732F426F6F742F6964652F2E2E2F2ED4
S113221C2E2F2E2E2F2E2E2F536F757263652F415A
S113222C524D434D335F4C4D33532F63616E2E63CC
S10F223C000800004F70656E424C540016
S1042248048D
S90300F10B
